:020000040000FA
:10000000831670308F001628C100030EC20004084A
:10001000C3000A08C4000B19C22144088A0043081F
:100020008400420E8300C10E410E090003019B00B3
:100030002730850004308600D730810024309800B6
:1000400019309900831290309800073085000030F5
:100050008600203084008001840A45300402031D9C
:100060002B280508073A0739B7008316203085008A
:100070008312A621E7308100A0308B008B13A70AE2
:100080000730A7052430A60033080739A5008C1ACD
:100090009528AA01A90129082B3E84000008A80080
:1000A0002708031D57282808031967286528033CDB
:1000B00003195E282708063C031D6128A81C672831
:1000C00065282808033C031D67288B20AA04A90A79
:1000D0002908083C031D4B28AA1BA6172A1B261714
:1000E000AA1A26162A1AA615AA19A5172A19251713
:1000F000AA1825162A18A5152430860033080739B2
:1001000085001A2225088500260886002708073C56
:1001100003198B173E28290882070134023404345E
:100120000834103420344034803418199E2998182B
:100130009E291A08A300523C031D22298C1E9E28CA
:1001400018199E2998189E291A08A300073C031C19
:10015000A1298C1EA92818199E2998189E291A08C9
:10016000A000073C031CA129A030840020088000C7
:100170008C1EB82818199E2998189E291A08A000C4
:10018000A1000319A1293C3C031CA129840A2008D1
:100190008000A00CA00C0F30A00521080339031D1E
:1001A000A00AA00D1E30A0058C1ED42818199E2967
:1001B00098189E291A08A1000319A1291F3C031CA5
:1001C000A129840A210880002308BA00BA0DBA0DBB
:1001D0001C30BA05B901A030BC000330BB00282296
:1001E000FF39031DA1295822FF39031DF3280630CA
:1001F00022222030B900A03084002030BB008C1EA9
:10020000FF2818199E2998189E291A088000840A28
:10021000BB0BFF28A030BC002030BB002822FF39D8
:10022000031DA1295822FF39031D12292030B907C7
:100230000318BA0A06302222A00BFB282308B700B5
:10024000A621A32954302302031D73298C1E2629BD
:1002500018199E2998189E291A08A300073C031C08
:10026000A129543022222308BA002222BA0DBA0D45
:100270001C30BA05B901A030BC000330BB007922A4
:10028000FF39031DA129A030840000082222840A1E
:100290000008A0002222A00CA00C0F30A00500082E
:1002A0000339031DA00AA00D1E30A005840A000812
:1002B00022222030B900A030BC002030BB007922BF
:1002C000FF39031DA129A030840000082222840ADE
:1002D000BB0B65292030B9070318BA0AA00B5B29AC
:1002E00006302222A3294B302302031D89298C1EAC
:1002F000772918199E2998189E291A080319A129E7
:10030000A3001F3C031CA1292308B40006302222AD
:10031000A32950302302031DA1298C1E8D291819F1
:100320009E2998189E291A08A300073C031CA1299E
:100330002308B70006302222A621A3291A08181282
:10034000181615302222B601B3013E283708BA002C
:10035000BA0DBA0D1C30BA05B901A030BC0003308B
:10036000BB007922FF39031DA629A03084000008B4
:10037000B800840A0008B500840A0008B400B60179
:10038000B3010800E73081000B11B30A3308A20063
:10039000A20CA20CA20C22081F393402031DDE2974
:1003A000B301B60A36083502031DDE29B601380846
:1003B00037020319DE293808B700A6213708BA002A
:1003C000BA0DBA0D1C30BA05360E0339BA07330818
:1003D000A200A20DA20DA20D22083839203EB900BC
:1003E000360EC039B9070318BA0AA030BC0008306D
:1003F000BB007922FF39031DF529A901A030290787
:1004000084000008A8003608033A0339A200031943
:100410000D2AA80CA80CA203072A0330A805290856
:100420002B3E840028088000A90A2908083C031DE7
:10043000FE2908000130A4000000A40B1C2A0000C3
:10044000000008008316981C222A831299000800D5
:10045000C001D222A0305A22FF390319382AC00A1B
:100460004008033C031D292A861000000610FF34B3
:100470003A085A22FF39031D2F2A39085A22FF3918
:10048000031D2F2A3B08BD003C08840000085A22A7
:10049000FF39031D2F2A840ABD0B462A06100000CF
:1004A00086140000061400008610000006100034B8
:1004B000D222A030BF000830BE000610BF1B0614B9
:1004C0000000BF0D861400008610BE0B5D2A831647
:1004D0000313061483120313861400000618BE03C8
:1004E00086108316031306108312031306103E08AA
:1004F0000800C001D222A0305A22FF390319892AEC
:10050000C00A4008033C031D7A2A8610000006102A
:10051000FF343A085A22FF39031D802A39085A222B
:10052000FF39031D802ADB22A1305A22FF39031D27
:10053000802A3B08BD003C08840083160313061480
:10054000831203130830BE00BF0D86143F10061837
:100550003F148610BE0BA42A3F088000840ABD0BFE
:10056000B22ABD2A83160313061083120313061042
:1005700000008614000086109D2A831603130610BF
:100580008312031306140000861400008610000076
:1005900006100000861400000614000086100000FB
:1005A00006100034831603138610061083120313FB
:1005B00086100614000006140000861400000610C1
:0605C00000008610080097
:02400E00303F41
:02401000FC3F73
:00000001FF
